:100000003EC0C4C157C056C055C054C053C052C0F2
:1000100051C050C04FC04EC04DC04CC04BC0040377
:1000200009041A03540069006C006C0020004800A9
:10003000610072006200610075006D001A036900C2
:10004000320063002D00740069006E0079002D00FD
:1000500075007300620012011001FF000008030424
:1000600031C60501010200010902120001010080F0
:10007000050904000000000000000100FF8E1124AB
:100080001FBECFE5D1E0DEBFCDBF10E0A0E6B0E0FF
:10009000EAE5FAE002C005900D92A636B107D9F75D
:1000A00010E0A6E6B0E001C01D92A939B107E1F762
:1000B00067D3D1C4A5CF85B7836085BF8BB7806474
:1000C0008BBF0895FF920F931F93CF93DF9360919F
:1000D0007F00662351F180917C00CCE0D0E0C81B0A
:1000E000D109CD57DF4F635080917B008D3279F07D
:1000F0008091660087FD11C0CE0165D38F3F09F462
:100100008FC0882309F489C090E080E008C08AE5A8
:1001100080936100683009F4A2C090E880E0909379
:1001200066008093600010927F008091610084FFE0
:1001300026C0809160008F3F11F1182F893078F52B
:10014000811B809360008091660080FD30C02BE4AD
:10015000F22E8F5F8093660087FD30C0112309F077
:100160004FC004E080E790E0612F81D2183019F091
:100170008FEF80936000F0926F00009361009AE02F
:1001800086B3857031F49150D9F7109280001092A7
:100190007A00DF91CF911F910F91FF90089518E0A1
:1001A000811B809360008091660080FFD0CF93EC2C
:1001B000F92E8F5F8093660087FFD0CFC0917D00BE
:1001C000D0917E0086FD32C0112399F01150DE01DE
:1001D000E0E7F0E0412F50E01F5F9A012F583F4FBA
:1001E0008D918193E217F307D9F74F5F5F4FC40FEB
:1001F000D51FD0937E00C0937D00012F0C5FB2CF3E
:1002000080E790E0612F2ED3182F893008F4A4C026
:100210008FEF809360000EE1AECF90E08FEF7FCF45
:100220008EE18093610090E08FEF79CF112309F385
:1002300011509E01A0E7B0E0612F70E01F5FAB019D
:100240004F585F4FF90184918D932F5F3F4FA41753
:10025000B507C1F76F5F7F4FC60FD71FCACF888121
:10026000807629F528E730E010927800898188238C
:1002700089F41092790030937E0020937D0090E8FD
:1002800022E08F81882321F48E81821708F447CFE2
:10029000822F45CF8530B9F08630F1F0883031F1CA
:1002A0008930A1F18A3059F190E820E0EACFCE01FF
:1002B0002DD3282F8F3F09F04DC0888187FD09C0BD
:1002C0008FEF90E02CCF8A818093800090E820E02F
:1002D000D8CF8E8190E023CF8B81813031F1823075
:1002E000D9F0833059F190EC20E0CBCF82E890E058
:1002F00090937E0080937D0090E821E0C2CF309300
:100300007E0020937D0090E821E0BBCF8A8180931E
:10031000820090E820E0B5CF88E690E090937E00E0
:1003200080937D0090EC22E1ACCF86E590E0909345
:100330007E0080937D0090EC22E1A3CF8A81882308
:1003400071F48EE190E090937E0080937D0090ECBC
:1003500024E097CF90E895CF082F0C5F03CF813032
:1003600061F0823009F0BFCF8CE390E090937E0083
:1003700080937D0090EC2AE184CF82E290E090931C
:100380007E0080937D0090EC2AE17BCFCF93CFB7A6
:10039000CF93B09BFECFB09B09C0B09B07C0B09B72
:1003A00005C0B09B03C0B09B01C09EC0DF93C0914D
:1003B0007C00DD27CD57DF4FB09B02C0DF91EBCF34
:1003C0002F930F931F9306B32FEF00FB20F94F934A
:1003D0003F9316B34FEF012700FB21F93BE031C0FB
:1003E0004E7F012F16B3216028C0102F4D7F226051
:1003F000000006B329C04B7F2460012F000016B314
:100400002BC016B3477F28602AC04F7E06B32061F9
:100410002CC04F7D16B320622FC04F7B06B32064E3
:1004200032C0422706B349934FEF0000102710FB5C
:1004300020F916B31570A9F1297F91F2012700FB6D
:1004400021F906B3237F89F23150F0F1102710FB18
:1004500022F916B3277E79F2012700FB23F92F7CBE
:1004600081F206B3102710FB24F92F7971F200C036
:1004700016B3012700FB25F92F7359F200C006B30C
:10048000102710FB26F9223040F200C016B30127D6
:1004900000FB27F9243028F64F77206816B30000B8
:1004A000F9CF3B503195333010E41ABFB8F0C31B7D
:1004B000D0400881033C41F10B3431F11981412FC7
:1004C0001F7720917A00121731F4093691F10D321D
:1004D00079F0013E69F02227209381003F914F91EE
:1004E0001F910F912F91DF91CF91CFBFCF91189591
:1004F000009381003F914F911F910F912F91DF91B8
:10050000CAB7C6FD46CFF0CF00918100002331F37A
:1005100010917F00112349F534304AF130937F0068
:1005200000937B0010917C003BE0311B30937C00FA
:100530001EC000917F000130C4F40AE530916100D3
:1005400034FD17C000936100CFE6D0E016C0052748
:1005500010E008BB1FC0052722C0052727C00527BC
:100560002CC0052710E008BB33C04AE503C042EDAC
:1005700001C0432FC4E1D0E032E017B31560C09A48
:1005800008B317BB5F9355E020E820FF052708BBA1
:10059000279517951C3FD8F620FF0527279508BB00
:1005A00017951C3FC0F620FF05272795179508BB18
:1005B0001C3F98F620FF0527279517951C3F08BB81
:1005C00070F600C0499120FF052708BB27951795B5
:1005D0001C3F38F620FF0527279508BB17951C3FC1
:1005E00038F520FF05272795179508BB1C3F10F508
:1005F00020FF0527279517951C3F08BBE8F4242FFB
:100600003A9519F60A7F5F9108BB00C010918000EF
:10061000C651D04011F010937A0010E41ABF016067
:1006200017B31A7F402F4A7F08BB17BB48BB56CF72
:100630000527D3CF0527D8CF0527DDCFA82FB92F82
:100640008FEF9FEF41E050EA615070F02D9138E05C
:10065000722F782796958795269570FF02C084277C
:1006600095273A95A9F7F0CF809590950895E6DF04
:100670008D939D930895882319F4B99AC19808958C
:10068000B998C19A0895E0916400F091650031979E
:10069000F1F7882359F0BD98C59AB59BFECF80919C
:1006A0006200909163000197F1F70895BD9AC59893
:1006B000F6CF81E0E8DF80E0E6DF089580E0DBDF71
:1006C00081E0E1DF81E0D7DF08950F931F93CF939F
:1006D000DF93082F10E0C7E0D0E008C081E0CBDF57
:1006E000E8DF21978FEFCF3FD80789F0C8010C2EA4
:1006F00002C0959587950A94E2F780FDEFCF80E0E0
:10070000BADFD7DF21978FEFCF3FD80779F781E0A6
:10071000B2DF81E0B8DF16B380E0B5DF1695109543
:10072000812F8170DF91CF911F910F910895FF92DA
:100730000F931F93F82E81E09EDF80E0A4DF17E087
:1007400000E081E0A0DF000FB199016080E09BDF55
:100750001150B8F7FF2051F480E08DDFAADF81E06F
:100760008ADF802F1F910F91FF90089581E083DF32
:10077000A0DF81E080DF802F1F910F91FF9008950F
:100780002EE088E190E00FB6F894A89581BD0FBEE9
:1007900021BDB998C19ABD98C59A10926D0010926A
:1007A0006C0088B38A7F88BB87B3856087BB80E491
:1007B0009CE90197F1F787B38A7F87BB7CDC78944B
:1007C000A89580DCFDCFEF92FF920F931F93CF93FC
:1007D000DF93E82E292FF62E80916700813091F566
:1007E00000916C0010916D00862F90E0081719079A
:1007F00008F4F02EFF20A1F08E2D922F9C01E9012C
:10080000899163DF9E012E192F15D0F301501040FE
:10081000FA940F191109F39410936D0000936C0072
:1008200080916E0081FF06C080916C0090916D00F8
:10083000892BB1F08F2DDF91CF911F910F91FF90F8
:10084000EF9008958E2D60E070E04F2D50E0FCD0C9
:100850008F2DDF91CF911F910F91FF90EF90089511
:100860002DDFE8CFCF92DF92EF92FF920F931F938D
:10087000CF93DF93C82E292FD62E80916700813029
:10088000E1F5E0906C00F0906D00862F90E0E816A6
:10089000F90608F4DE2CDD20E1F08C2D922F9C016E
:1008A0008901E701219780E009F481E040DFF80148
:1008B00081938F018E2F8C198D15A0F30894E10878
:1008C000F108DA94ED18F108D394F0926D00E092FB
:1008D0006C0080916E0081FF06C080916C00909149
:1008E0006D00892B89F08D2DDF91CF911F910F9194
:1008F000FF90EF90DF90CF9008958C2D60E070E036
:100900004D2D50E0A1D0EFCFD9DEEDCF1F93CF9387
:10091000DF93EC0188E690E090937E0080937D0069
:100920002981223009F456C0233070F1233009F4B4
:1009300067C0283008F03EC01C81110F8A8180FDFD
:100940001160898180FD04C081E095DE81E09BDE3D
:1009500080E091DE80E097DE812FB7DE882309F406
:100960005FC081E0809367002E813F8130936D00EE
:1009700020936C00898180936E0081FF4DC0232BF2
:1009800009F447C08FEF17C02223C9F0213091F43A
:100990006AE770E044E050E04ED084E0DF91CF9110
:1009A0001F910895969587959093650080936400B4
:1009B000892BF1F080E0DF91CF911F9108958A811A
:1009C000809368008B818093690082E0DF91CF91F2
:1009D0001F9108958A819B819093630080936200A8
:1009E000009701F781E090E09093630080936200AC
:1009F00081E090E0909365008093640080E0DBCF1D
:100A0000809167008093680081E0DF91CF911F9112
:100A1000089554DE2E813F81232B61F28FEFCBCFDF
:100A200082E08093670010926D0010926C0046DEA9
:100A30002E813F81F1CFFB01DC0102C005900D92B8
:100A400041505040D8F70895DC0101C06D934150EA
:0A0A50005040E0F70895F894FFCF3E
:060A5A00FF5A0A0005002E
:00000001FF
